:020000040000FA
:020000000528D1
:06000A008316073085009B
:100010008601831285018601050882071628232898
:100020001A2823282C2816282C281A283E20352068
:1000300047200C287420502059207D2059206B2007
:10004000742062200C285920502059207D205920EE
:100050006B20592062200C2874206B2074206220B1
:100060007420502074207D200C280D309C00061434
:10007000862006108F209C0B372808000D309C002E
:100080008614862086108F209C0B402808000D3097
:100090009C000615862006118F209C0B492808001D
:1000A00008309C000614AA200610B3209C0B52288E
:1000B000080008309C008614AA208610B3209C0BF0
:1000C0005B28080008309C000615AA200611B32002
:1000D0009C0B6428080008309C0006149820061029
:1000E000A1209C0B6D28080008309C0086149820E5
:1000F0008610A1209C0B7628080008309C0006156D
:1001000098200611A1209C0B7F28080031308C001C
:1001100008308D008D0B8A288C0B8828080032301F
:100120008E005C308F008F0B93288E0B9128080077
:100130002C308C0007308D008D0B9C288C0B9A285E
:10014000080035308E0058308F008F0BA5288E0B9D
:10015000A328080034308C0009308D008D0BAE28A8
:100160008C0BAC28080035308E0055308F008F0B7B
:08017000B7288E0BB52808002A
:00000001FF
